:1000000000308A00942800008C1E04281808A000E4
:100010001A08F800A01C0E28181218168A110A12C5
:10002000DF282208303C031D2228BD113D0883161D
:100030008700831287113D103D08831687008312C5
:1000400007142E28BD113D088316870083128715DB
:100050003D103D08831687008312071023080F39CF
:10006000F700770EC000F030C00524080F394007B4
:10007000B900BA01390DBF003A0DC000BF0DC00D67
:10008000FC30BF05C00CBF0CC00CBF0CC00C3F083F
:100090009500C00C400C3039F7001708CF397704B1
:1000A00097002508303C031D6228BD123D088316C9
:1000B0008700831287123D123D0883168700831242
:1000C00007166E28BD123D08831687008312871617
:1000D0003D123D08831687008312071226080F3948
:1000E000F700770EC000F030C00527080F39400731
:1000F000BB00BC013B0DBF003C0DC000BF0DC00DDF
:10010000FC30BF05C00CBF0CC00CBF0CC00C3F08BE
:100110009B00C00C400C3039F7001D08CF39770424
:100120009D008A110A124929840183131F30830517
:10013000403083169900A2309800903083129800C6
:1001400083161F149F141F159F1107309C008312E4
:10015000A001FF30BD0083161F149F141F159F11AF
:10016000803087008312BD00F03083168600003097
:10017000850081130F30831286003D113D088316E0
:100180008700831207110C309700BD103D088316BD
:100190008700831287100C309D000030F80004386F
:1001A0009200FF3083169200831295019B01870114
:1001B0008316861183128611B601B70104287808C8
:1001C000A10036080319F128013A0319F828033A67
:1001D00003190129013A03191029073A03192029A3
:1001E00050292108533C031DF7280130B60052293D
:1001F0002108533C031DFF280230B6000029B60138
:100200005229223037078400831321088000B70A5F
:100210003708053C03180F29B7010330B6005229EF
:100220002C30370784008313210880008009B70A27
:100230003708053C03181F29B7010430B6005229BE
:100240002108453C031D4E29B801BE013E08053C6E
:10025000031C3C2922303E07840083130008BF00A2
:100260002C303E078400831300083F0203193A290B
:100270000130B800BE0A2629B808031D4A29831692
:1002800006110430831286068316061083120614A4
:1002900011284E298316061083120610B601522922
:0802A000B6015229DE286300BB
:02400E00723FFF
:00000001FF
